:100000004AC06FC06EC06DC06CC06CC06AC069C0B1
:1000100068C067C066C065C064C063C062C00000DD
:1000200000000000000000000000000000000000D0
:1000300000000000000000000000000000000000C0
:1000400000002167B1FF030405070A0E1319212BD5
:10005000364353657990AAC6E6FFFFFFFFFFFFFF17
:10006000FFFFFFFFFFFFFFFFFFFFFFFFFF0000009D
:100070000000000000000000000000000000000080
:10008000000008121C2834414E5C6B7C8FA3B8CF53
:10009000E6FFFFFFFF0011241FBECFE5D1E0DEBF6A
:1000A000CDBF20E0A0E6B0E001C01D92A238B207AB
:1000B000E1F7E1E6F0E085E5808781E08383148263
:1000C00012828683118288E081878FE48287612C87
:1000D000ECE6F0E08DEF87838EEF8583712C78D08E
:1000E000ABC08ECF189525B7277E25BF29B72260D4
:1000F00029BF21E022BF019728F020E188952150F7
:10010000E9F7F9CF089588EE93E0EDCF369A369966
:10011000FECF85B10895811104C01BBC19BC18BC69
:100120000895815090E0FC01E25EFF4FE491EBBD49
:10013000FC01EA5BFF4FE491E9BDFC01E259FF4F8E
:10014000849188BD08950F931F93CF93C82F8B017F
:10015000CC2369F08AE0DFDFC801C5DF1BBC19BC16
:1001600018BCC801C0DFC801BEDFC150F1CFCF91BC
:100170001F910F910895CF93DF93D82F64E170E022
:100180008AE0E1DF84EF91E0AEDF8D2F64E648D0B6
:10019000CAE06C2F45D0892F68EC70E0D4DFB3DF64
:1001A0008D2F6C2F3DD0D92F3BD0892F68EC70E07C
:1001B000CADFA9DF68EC70E08D2FC5DFA4DF64E142
:1001C00070E08AE0C0DF84EF91E0DF91CF918BCFC8
:1001D00083EA87B986EC86B93699FECF369A369986
:1001E000FECF85B18095882E8FEF8DBD80E68CBDCA
:1001F0008FE384BB8BE187BB88EE88BB81E083BF44
:1002000091EA9ABD80BF85B7806285BF789497B91F
:1002100086EC86B98CE291E066DF78DFACDFFACF5E
:10022000991B79E004C0991F961708F0961B881F48
:0C0230007A95C9F780950895F894FFCFE7
:00000001FF
